:020000040000FA
:0600000000008A01B72D8B
:08000800F0000308F1000A08F2
:10001000F2008A0183120313083081070B115C2060
:1000200019205C2072088A0071088300F00E700E9F
:10003000090087013F200310F70DF71E0800741C0C
:100040002D28203084001930F8008413000884170C
:100050008000840AF80B25287410A0308400013039
:10006000F700F90803193628F9030319F414FA0BF9
:1000700008006430FA00FB08031DFB0308004B2056
:100080004B204B204B204B20043085000030850056
:100090007708870008000530F800000DF600F60D1F
:1000A000F60D0030F60D0318023885000138850082
:1000B000F80B5128840A08000408F3067306F306B7
:1000C00084000800F5186B2875186E28751D080047
:1000D0007220800608007220800408007220FF3A17
:1000E000800508003F0884000310840D840D8407F8
:1000F000203084074008840700308A003E088207C9
:10010000103408340434023401341930C100203072
:1001100084008009840AC10B892808001F30A000D0
:10012000A100A200A300A400A500A600A700A800AB
:10013000A900AA00AB00AC00AD00AE00AF00B0005B
:10014000B100B200B300B400B500B600B700B8000B
:1001500008001F30F5188000751880017519800699
:1001600008006220BD20BD20BD20BD200800622007
:10017000C120C120C120C1200800840A840A840A49
:10018000840A840AF518800475198006751880059C
:100190000800C001BF01B120C00AB120C00AB120CF
:1001A000C00AB120C00AB1200800C0017220A920F5
:1001B000840AA920840AA920840AA920840AA920E3
:1001C0000800BF017220A92005308407A92005304E
:1001D0008407A92005308407A92005308407A920B9
:1001E00008003330C500450884000008840A840AEA
:1001F000840A840A840A8000C50345081F3A031D47
:10020000F328A001A101A201A301A4010800253047
:10021000C500450884000008840384038403840324
:1002200084038000C50A4508393A031D0929B40131
:10023000B501B601B701B80108003730C50045085F
:1002400084000008840A8000C50345081F3A031D86
:100250001F29A001A501AA01AF01B40108002130A6
:10026000C50045088400000884038000C50A4508CD
:10027000393A031D3129A401A901AE01B301B80126
:1002800008001930C500203084008012800C840AD8
:10029000C50B452908001930C50020308400031023
:1002A000800D840AC50B4F2908006220C703073060
:1002B000470503198329C71D61293E0A3E19030119
:1002C000BE00461C68290430BE08031D3E03BE0064
:1002D000471E6E293F0A3F190301BF00C71E75293B
:1002E0000430BF08031D3F03BF00471F7B29400A9E
:1002F00040190301C000C71F82290430C008031D34
:100300004003C000552908002008C2003408A0009E
:100310003808B4002408B8004208A4002108C2002C
:100320002F08A1003708AF002908B7004208A9002C
:100330002208C2002A08A2003608AA002E08B60029
:100340004208AE002308C2002508A3003508A50016
:100350003308B5004208B3002608C2003008A600E2
:100360003208B0002808B2004208A8002708C200DE
:100370002B08A7003108AB002D08B1004208AD00E2
:1003800008000A248A01C600C61B122A461B022A3C
:1003900001308A00CF30460703188A0A8200C1293B
:1003A000E42AE72A892AAB2AB12AAE2A232ABB2AC1
:1003B000BB2ABB2A6E2AC62AC62AC62AB42AB72A4C
:1003C000B92A882B8A2B102B0E2B122B142B162BB1
:1003D000182B3F2A442A4A2A502A542A582A5C2A8F
:1003E000A92A0A2B3D2ADB2BE22BE92BF02BF72B3A
:1003F000EA2AED2A622AA12BA32BAC2BFE2BB12BD0
:10040000BC2BC92B5E2302308A000A304607031832
:100410008A0A8200DC2AD42AE02AD82A7C2B7F2B65
:10042000F72AFB2A0A248A01C700461B662AC61A35
:10043000702A460C0F39031D1F2A4C23C129FF3E89
:10044000031D252A4C236220C129FF3E031D2A2AB1
:100450005521C129FF3E031D2F2AF5151A2BFF3EFA
:10046000031D342AF5111A2BFF3E0319FF2AFF3E04
:100470000319042BFF3E0319922A8421C129342435
:100480007220A9203B24C1293424BF017220B1204D
:100490003B24C1293424C0017220B7203B24C12948
:1004A0003424C9203B24C1293424D5203B24C1292C
:1004B0003424E1203B24C1297220F41100050319E2
:1004C000F415C129F411051EF415C129C61A6823B3
:1004D00046081F39FD004708FC00C1297223C129C5
:1004E0005E234611460803197C2AFF3E03197F2A22
:1004F000FF3E0319832A112C47088000C1294708B1
:1005000012248000C129F41547080006031DF411C8
:10051000C129F41C892AF41074143D08F9007418D8
:100520008F2AC1296430FA004708FB00F411C7087C
:100530000319FB17FB080319C129051E972AC708D1
:100540000319FB17FB080319C129051A9F2AF41583
:10055000C1292D24C1290130F500C1290430F5003D
:10056000C1290230F500C12903018F20C1298E2045
:10057000C1298520C129460803393E3E8400043044
:100580008008031D00038000CF2AC12946080339D3
:100590003E3E8400800A0008053A03198001F415E4
:1005A0008008031DF411C1298003031DC129F02A0D
:1005B000800A031DC129F02AF415800BF411C1290A
:1005C000F415800FF411C129F41DC129F02AF41D7E
:1005D000F02AC129741EC129F02A741EF02AC129EB
:1005E0000A248A018039031D0A248A01C1290008CE
:1005F000C700F5151A2B0008C700F5111A2B643037
:10060000FA004708FB00C1296430FA0047081224A9
:10061000FB07C129FB08031DC129F02A1D21C1299F
:100620002F21C129F120C1290721C1294B21C1292D
:100630004121C1293424FF01203047023F39FE0007
:100640000310FE0DFE0DFE070318FF0A4230FE07E1
:100650000318FF0A0430FF070530C7000430F519FE
:10066000BF00F51DC001722048238A01F5188004DF
:1006700075198006FF3A75188005FE0A0319FF0AEE
:10068000F519BF03F51DC00AC70B332B3B24C12945
:100690007F088A007E0882004708BF000739C00033
:1006A000BF0CBF0C3F0C0739BF004708BE00460C0B
:1006B000BE0DBE0D3E0D0739BE00080046080739C5
:1006C000393E8400C60CC60C460C0739C60008002B
:1006D000430884007C088000840A7D088000040AA6
:1006E000C3000800430384000008FD0084030008E1
:1006F000FC000408C300080000088C23C12904087A
:10070000C7009823C5004708840045088000C12918
:10071000CD23C129D423C129C5004408840045083C
:100720008000C40A4408EB3AC9300319C400080029
:100730004408C93AEA30031D4403C4008400000899
:1007400008009823C1299823CE009823CF004E0893
:100750008C234F088C23C12998238C2345088C2394
:10076000C1299823CE009823CF004E088C234F0830
:100770008C234E088C23C1299823CE009823CF00C8
:100780009823D0004F088C234E088C2350088C23CC
:10079000C129982306248C23C1293E088C233F08B5
:1007A0008C2340088C2308009823C0009823BF00A6
:1007B0009823BE0008009823CD0098234D060624F8
:1007C0008C23C1299823CD0098234D0703248C2323
:1007D000C1299823CD0098234D0203248C23C129DD
:1007E0009823CD0098234D0506248C23C1299823F6
:1007F000CD0098234D0406248C23C1299823FF3A69
:1008000006248C23C129741203187416F4110319D9
:10081000F41508007D088A007C08FC0A0319FD0A0B
:100820008200112CCA000310C80CC90C031C1B2C1D
:10083000A130C806C9064808490403192D244908EF
:100840004807CB01CC01CC17CA0C0318CB07CB0C43
:10085000CC0C031C242C4B080800010803192D2C78
:10086000C900FF3AC80008003E08CE003F08CF008C
:100870004008D00008004E08BE004F08BF005008D6
:10088000C000080000340034003400340034043464
:1008900004340434003404340A340A340034003498
:1008A00000340A341F340A341F340A340F34143429
:1008B0000E3405341E3419341A3404340B34133412
:1008C000083414340D3412340D340C340C34043424
:1008D0000834003402340434043404340234083458
:1008E000043404340434083415340E341F340E3404
:1008F0001534043404341F340434043400340C3408
:100900000C3404340834003400341F340034003410
:100910000034003400340C340C3401340234043418
:10092000083410340E341334153419340E340434AE
:100930000C34043404340E341E34013406340834C8
:100940001F341E3401340E3401341E3406340A348C
:100950001F34023402341F3410341E3401341E3468
:10096000063408341E3411340E341F340234043477
:10097000083408340E3411340E3411340E340E346D
:1009800011340F3402340C340C340C3400340C3475
:100990000C340C3400340C34043408340234043481
:1009A00008340434023400341F3400341F3400345B
:1009B000083404340234043408340E34113402345C
:1009C000043404340E341534173410340E34043423
:1009D0000A341F34113411341E3409340E340934EE
:1009E0001E340F341034103410340F341E340934D4
:1009F000093409341E341F3410341E3410341F34AB
:100A00001F3410341E34103410340F3410341334A7
:100A100011340F34113411341F34113411340E34A5
:100A20000434043404340E340134013401341134F8
:100A30000E34133414341834143413341034103482
:100A4000103410341F3411341B3415341134113464
:100A5000113419341534133411340E341134113463
:100A600011340E341E3411341E34103410340C344E
:100A70001234163412340D341E3411341E3414342E
:100A800012340F3410340E3401341E341F34043445
:100A900004340434043411341134113411340E3458
:100AA0001134113411340A3404341134113415342E
:100AB0001B34113411340A3404340A34113411341F
:100AC0000A340434043404341F3402340434083443
:100AD0001F34073404340434043407341034083425
:100AE0000434023401341C340434043404341C341B
:100AF00004340A3411340034003400340034003437
:100B000000341F3487011930F800A0019F25F80B2D
:100B1000862D8316031300308F00831203130130D8
:100B2000F70087001930F8000130A0009F25F80B6E
:100B3000962D0310770D771A0130F700922D0230B1
:100B4000A00B00398500A000B225200801388500DF
:100B5000B2250430850077088700B2250030850073
:100B6000B2250800FF30FF3E031DB32D08006400CE
:100B70000730990083160313910170308F00033002
:100B80008100F83085003030950083120313203047
:100B900084008417800184138001840A841FC92D76
:100BA00083160313E030870083120313851E822D02
:100BB000A030F3000130F700F4140530FD00EC30F4
:100BC000FC00C930C400B930C3000130BD0008309A
:100BD0008100A0308B00C12921342B340234C6346B
:100BE0006E34E634AE34A4340934A8341D345034A1
:100BF000E534FC34C534F33440340234C634FA34BA
:100C000040340234C7347D3440340234C734B43401
:100C100040340234C834193440340234C8344634C1
:100C200040340234C8347C3440340234C834923402
:100C300040340234C934573440340234C934CB34DC
:100C400040340234C934FD3440340234CA344534AB
:100C500040340234CA346D3440340234CA349934D6
:100C600040340234CB341C3440340234CB344A3464
:100C700040340234CB344E3440340234CB3452341A
:100C800040340234CB34A83440340234CC341534EC
:100C900040340234CB34F63440340234CC345D3446
:100CA00040340234CC34A43440340234CC34E934FB
:100CB00040340234CD345E3440340234CD34B53463
:100CC00040340234CE340C3440340234CE34413417
:100CD00040340234CE34C334C534FC34E634AE344C
:100CE000E634FA34E7347D34E734B434E834193484
:100CF000E8344634E8347C34E8349234E934573408
:100D0000E934CB34E934FD34EA344534EA346D3423
:100D1000EA349934EB341C34EB344A34EB344E343B
:100D2000EB345234EB34A834EC341534EB34F63471
:100D3000EC345D34EC34A434EC34E934ED345E341A
:100D4000ED34B534EE340C34EE344134EE34C33487
:100D5000C63470342234C634AA340B34A734043475
:100D60000534A0345034E634EA34A0344934E6344F
:100D7000EA34A0344334E634EA34A0345034E63460
:100D8000EA34A0345234E634EA34A0344F34E63442
:100D9000EA34A0344A34E634EA34A0344534E63444
:100DA000EA34A0344334E634EA34A0345434E6342C
:100DB000EA34A0345334E634EA34A0342034E63440
:100DC000EA34A0344334E634EA34A0343334E6342D
:100DD000EA340B34A43408340F347034033414343C
:100DE000033414340334143403341434A434233457
:100DF00003340B34A43409348A3405348C34073476
:100E000005340F348034003484341D348134043488
:100E10008534153403340F348034403484341C3426
:100E2000833421348034C4348534143482342334FC
:100E300003340F348034803484341B3481341934C7
:100E400084345234803484348534133480341B34F5
:100E50008434923403340F348034C03484341A34EC
:100E6000813411348434533480344434853412341E
:100E7000803413348434933403340F348134003495
:100E800084345534803404348434953403340F343A
:100E900081340134843454348234E434803403346F
:100EA000843494348234603403340F348134023413
:100EB000843453348034DC34853412348034023446
:100EC000843493348034583484341A3403340F34E3
:100ED00081340334843452348034D434853413342C
:100EE00080340134843492348034503484341B345C
:100EF00003342234C73401340B34A43401340F34A6
:100F00000534803400341E3403348A340A34A43463
:100F10000F340334AD340534AF340534A634003413
:100F2000A0340434A434053420340134C734A53447
:100F3000A634043404340734093405340734033444
:100F40004834C7349A34C734B034043407340D34C9
:100F50000534073403344834C734A534C734B034B7
:100F60002234C73487340B348A340A340F340334C0
:100F7000A13400346134A4340334AD340534AE34C8
:100F80000534AF340534A934063468346034613430
:100F900024342C340234C734BB346134B1340034CB
:100FA0000234A5340034B13401340234A6340034A0
:100FB000B13402340234A7340034B134033402347F
:100FC000A5340434B13404340234A6340434B134C6
:100FD00005340234A73404340534A0340534E7342E
:100FE000FB340434A0340534E734FB3403342234B6
:100FF000C734BB340B3407340334B1340034023407
:101000000C34B134013402340D34B13402340234BE
:101010000E34B134033402340834B13404340234AD
:101020000934B134053402340A344834C734FB344B
:101030000B340F3403340534A434233482340034A5
:10104000833400348334203483342434823424348D
:1010500082340434833404348234203403348234BC
:10106000493482344B348234593482345B34823490
:10107000C9348234CB348234D9348234DB340334FF
:101080008234923403340F34C634AA34A434323454
:101090000F34053482349234033482348A348234F7
:1010A0009A34823452348234D23482349134823449
:1010B00093340334803492341A341B341C34823415
:1010C00051348234D334823453348234D134823430
:1010D000893482348B3482344A348234CA34823440
:1010E000993482349B3482345A348234DA3403346F
:1010F0008A340134C634AA34A43407348A340F3411
:10110000A63400340F3405341634E8348C340334F8
:101110002234C83484340B34AD340534AF34053450
:1011200007340B340F34A4340F34053480340034C6
:101130001A34803404341A3403341C3481340034B7
:101140001C340334A6340034A5340034A7340034EE
:101150000734083407340A3407340C3407340334B2
:101160000D34B63400340134C834A4348034A2348D
:101170001E3404341A341C34033405341E3403344E
:101180001734033417340334173403341734033457
:1011900016340334163403340F348034103484345A
:1011A0000D348434453485340534843485348034B6
:1011B000593484340B3484344334853403348434D4
:1011C000833403348234A23403340F348234A2349F
:1011D00009341E34043482349A3403340D340F3409
:1011E00005341E34033404348234203483342034F0
:1011F00083342434823424340534823418348334E0
:10120000183483341C3482341C3403340F34803457
:10121000A2341A341C34823461348234633482340C
:10122000E3348234E13482345834823419348234E1
:10123000D8348334193483341B348234DC3482341C
:101240005C3482341B34823410348334103483345D
:1012500014348234143403341734043482345A344A
:10126000823499348234DA3482349B3482349A342E
:101270000534823462348234A1348234E2348234DC
:10128000A3348234A23403341734043482349A34BD
:1012900005348234A234033417340334173403344E
:1012A0001734033417340334173403340B340F3436
:1012B000053482344934823451348234893482345E
:1012C000913482344A348234523482348A348234BF
:1012D00092340334A4340B34A0341934A0340134D0
:1012E000A1340134A23401348A3405348C340A34F4
:1012F000AB3405340234C93495344B34C9349E348C
:10130000AB3404340234C934A7344B34C934B03458
:10131000AB3403340234C934C2344B34C934B93425
:1013200003342234C93478340B34B03400340234FA
:10133000C934803418344034C9348034B034033470
:101340000234C934803419345034C9348034B1344F
:1013500000340234C934883417344134C9348834F1
:10136000B13403340234C934883416345134C934A6
:101370008834B23400340234C934903414344234E2
:10138000C9349034B23403340234C934903415343F
:101390005234C93490340F340534A4340C348A34B4
:1013A0000A348C3406341534803410341A3404343E
:1013B000823490340534033415348034003484345A
:1013C0001D340434823490340534033415348034AD
:1013D00080341B340434823490340534033415349F
:1013E0008034203484342D340434823490340534F1
:1013F00003342234C934D3340B3405340F34A434C9
:101400000F34813400341A3403341C3403348034F0
:1014100004341A3403341C340334823408348234E0
:101420000C348334083483340C3403348234103461
:1014300082341434833410348334143403348234C7
:10144000183482341C348334183483341C34033409
:10145000813420341A3403341C340334803424346B
:101460001A3403341C34A43432340334A4340F3417
:101470001F34033414340334143403341434033465
:101480001434A434323403340B34A4340F3405340C
:101490000F3483342434033404341034823400345D
:1014A000EA34953482344934EA34953482349234BF
:1014B0000334103482340034EA34953482344934AD
:1014C000EA3495340334103482340034EA349534E9
:1014D00003341034033405340B34A4340F3405348E
:1014E0000F3482340034033404341034833424340D
:1014F000EA3495348234DB34EA34953482349234DD
:101500000334103483342434EA3495348234DB34A5
:10151000EA3495340334103483342434EA34953473
:1015200003341034033405340B341D341E341F349B
:101530000B340F34A4340934053482349434033426
:1015400082349334823453348234D33482348B34AF
:1015500082349B340334803492341A341B34823402
:101560005A3482344A348234DA348234CA3403340A
:101570001434823494340334143482349434033471
:10158000143482349434803400341F34043482346C
:1015900000348234203483340034833420340334E0
:1015A0000534143482349434803400341F340334CA
:1015B0000434823494348234903403348234933447
:1015C00082349034823450348234D034823488343B
:1015D00082349834033482349234803490341A3410
:1015E0001B3482345834823448348234D8348234C0
:1015F000C834033405340F34823400348234203448
:1016000083340034833420340334153403341534E4
:10161000033415340334153403340F3482344C341A
:1016200082345C348234CC348234DC3403340F347E
:101630008234943403340B340F340534A4340E3420
:1016400080340034EA34953403340F348034493420
:10165000EA34953403340F3480349234EA349534C8
:1016600003340F348034DB34EA34953403340F34DC
:1016700081342434EA34953403340B34A0340534F3
:101680001434183417348334243403344834CB34BA
:1016900040340B34EB345634CB346934EB345634A9
:1016A000CB349334EB345634CB347E340F3405349E
:1016B000AC3408346434A4340834643425346C34D1
:1016C00080341034A03401348A3404348C34063429
:1016D0000B341C34033419346034663425346E34CE
:1016E000B63404340234A034FF34B6340034023447
:1016F000A03401342234CB3469340B341B3403342A
:1017000015346034653425346D34B5340434023412
:10171000A034FF34B53400340234A0340134223410
:10172000CB347E340B341A340334153460346634CD
:1017300025346E34B63404340234A034FF34B63465
:1017400000340234A03401342234CB3493340B34CB
:10175000A43407346434AC340A34643425346C342F
:1017600010340334043480342034EB34E034EB346C
:10177000E034EB34E034EB34E034EB34E034033485
:10178000033480346134EB34EB34EB34EB34EB343E
:10179000EB34EB34EB34EB34EB340334033482348A
:1017A000A234033482349A340334823492340334BE
:1017B00082348A34033482348234033403340B3465
:1017C00084340D348434453485340534843485348C
:1017D000033409340B3484340B3484344334853477
:1017E000033484348334033409340B34A4340A348A
:1017F0000F3403348A3403348C3404340534833492
:101800002434AB340334A4340A34EC342334A43405
:1018100005346434AC340C34643425346C34EC3426
:1018200030342234CC340F340B34A4341934103413
:101830000334053483342434AB340434A4340A34FC
:10184000EC3430340B34B334003402341F34B3344A
:10185000013402341E34B334023402341D340B34E8
:10186000EC344134EC344134EC344134EC34413424
:10187000EC344F34EC344F34EC344F34EC344F34DC
:101880000B34B334003402341434B334013402342E
:101890001734B33402340234183403340B34B33401
:1018A000003402341534B334013402341634B33402
:1018B00002340234193403340B34A034013460345C
:1018C000A83404346034253468340F340534A43427
:1018D00003346434AC340734643425346C348034D9
:1018E00000341A34EC3490341534EC349A34153412
:1018F000EC3490341534EC349A341534EC349034A0
:101900001434EC349A341434EC3490341434EC340D
:101910009A341434EC3490344834CC3474340B346A
:1019200003341634033416340334163403341634B3
:1019300003340B34033417340334173403341734AB
:101940000334173403340B34A03403346034A83424
:1019500006346034253468340F340534A434033439
:101960006434AC340834643425346C34803400344A
:10197000803400341C34813400341C3403340F347C
:10198000803448341C348034C8341C3403340F345D
:10199000803490341C3403340F34803458341C3475
:1019A0008034D8341C3403340F34803420341C3455
:1019B000813420341C340334173403341734033493
:1019C00017340334173403344834CC34BF340B3465
:1019D00021340534A4340234A0340134A134013458
:1019E000A2340134803492348A3405348C340A347D
:1019F0000F3407340334ED3401342234CC34F8345A
:101A00000B346034653425346D34613466342534E8
:101A10006E346234673425346F34B53400340234A4
:101A2000ED342C34B53404340234ED343034B6346F
:101A300000340234ED343434B63404340234ED343A
:101A40003834B73400340234ED343C34B734043421
:101A50000234ED3440340B34ED34443468340B3408
:101A6000ED344A3468340B34ED34443469340B3487
:101A7000ED344A3469340B34ED3444346A340B3475
:101A8000ED344A346A340B34ED345534AB3402341B
:101A900063340B34ED345534AB340234B334013495
:101AA0000234A334FF3463340B34A434013464347B
:101AB000AC340834643425346C340B340F34A4341F
:101AC00002346434AC340634643425346C348034E9
:101AD0000034ED349C340D34ED34A8340D34ED3441
:101AE0009C340D34ED34A8340D34ED349C340E3474
:101AF000ED34A8340E34ED349C340E34ED34A83477
:101B00000E34ED349C340934ED34A8340934ED340A
:101B10009C340934ED34A8340934ED349C340A344F
:101B2000ED34A8340A34ED349C340A34ED34A8344E
:101B30000A34ED349C340B34053407340334043454
:101B400007340C340134CD349C34043408340B3461
:101B5000053407340334043407340834B53404340A
:101B60000134CD34A8340C340B34A43428340F346D
:101B70000534A63400341E340334A73404341F342F
:101B80000334A63404341E340334A53400341D3425
:101B90000334A53404341D340334A73400341F3413
:101BA00003340434A034FF34A4340034ED34DE3480
:101BB000073403344834CD34D6340B34A9340334D9
:101BC00041340234CD34F43441340234CE34003460
:101BD000A7340034A93402344934A7340434AD3472
:101BE0000534AE3405340B34A6340034A934023441
:101BF0004934A6340434AD340534AF3405340B34E1
:101C0000A5340034A93402344934A5340434AF3443
:101C10000534AE3405340B34A4340A34053482342C
:101C200094340334143482348C3482345434823403
:101C3000943482349C348234D43403341434823463
:101C4000A43483341434823494348234843482341B
:101C50001434033414340334823494341434033489
:101C6000823494341434033482349434143403347A
:101C70001434033414340334143403341434033468
:101C80000B340F34A73404340534A0343534E6342F
:101C9000EA34A0343434E634EA34A0343334E6345D
:101CA000EA34A0343234E634EA34A0343134E63451
:101CB000EA340F340534A4341934053482348234C0
:101CC0000334A434153416348234813482344234DB
:101CD00082348234823483348234C2340334A43470
:101CE000113416348234843483340234823482349E
:101CF00082348034823402340334A4340E341634F3
:101D00008234813482344234823482348234833463
:101D10008234C234033482348234A4340A34163414
:101D20008234813482344234823482348234833443
:101D30008234C234033482348234A43409341634F5
:101D40008234813482344234823482348234833423
:101D50008234C2340334823482340334A4340834E9
:101D60001634823482340334163482348234033499
:101D7000A4340634163403341634033416340334CE
:101D8000163403340B340F340534A4340C348A3441
:101D90000A348C34063416348034823484340B3460
:101DA000033416348034823484344B340334163490
:101DB000803482348434433403341634803482349F
:101DC0008534433403341634803482348534033408
:101DD0000334163480348234853483340334163427
:101DE000803482348434833403342234CE34CB348C
:021DF0000B34B2
:02400E00E43399
:1042000020004C004500440020004300750062007F
:1042100065002000560031002E0030002E003400D2
:10422000200043003300200061006E0069006D0033
:104230006100740069006F006E007300200031009F
:1042400035002D00300031002D00320030003100EB
:1042500031002000200070006900630070007200CF
:104260006F006A0065006300740073002E006F0029
:10427000720067002E0075006B00200020002800EF
:1042800063002900200032003000300039002D008A
:104290003200300031003100200050006500740011
:1042A0006500200047007200690066006600690032
:0842B000740068007300200097
:00000001FF
